:0200000480007A
:100000006F00C004732F2034930F8000630AFF0336
:10001000930F90006306FF03930FB0006302FF038A
:10002000170F0080130F0FFE63040F0067000F000F
:10003000732F203463540F006F004000136E9E53E3
:10004000171F00002320CFFD6FF09FFF732540F1A5
:100050006310050073251030635805000F00F00F82
:10006000130E100073000000130E00009702000032
:10007000938282F973905230735020307350303035
:1000800073504030970200809382C2F7638C020065
:10009000739052109302B01A739022307323203061
:1000A000E39E62F873500030970200009382420191
:1000B00073901234732540F17300203097200000B4
:1000C000938040F483810000930EF0FF130E200014
:1000D000639CD123972000009380C0F2838110009D
:1000E000930E0000130E30006390D1239720000080
:1000F000938040F183812000930E00FF130E400097
:100100006394D121972000009380C0EF8381300059
:10011000930EF000130E50006398D11F972000003B
:10012000938070EE8381D0FF930EF0FF130E60007A
:10013000639CD11D972000009380F0EC8381E0FF49
:10014000930E0000130E70006390D11D97200000E5
:10015000938070EB8381F0FF930E00FF130E8000FD
:100160006394D11B972000009380F0E98381000005
:10017000930EF000130E90006398D11997200000A1
:10018000938040E8938000FE83810002930EF0FF8D
:10019000130EA000639AD11797200000938080E689
:1001A0009380A0FF83817000930E0000130EB000B7
:1001B000639CD115130EC0001302000097200000AD
:1001C000938050E48381100013830100930E00FF9D
:1001D000631CD3131302120093022000E31052FE9B
:1001E000130ED00013020000972000009380A0E1BE
:1001F000838110001300000013830100930EF000B0
:100200006314D3111302120093022000E31E52FC68
:10021000130EE0001302000097200000938080DEA0
:1002200083811000130000001300000013830100FD
:10023000930E0000631AD30D1302120093022000E4
:10024000E31C52FC130EF000130200009720000084
:10025000938050DB83811000930E00FF6396D10BD7
:100260001302120093022000E31252FE130E00014B
:1002700013020000972000009380E0D813000000D4
:1002800083811000930EF0006390D10913021200D5
:1002900093022000E31052FE130E1001130200001F
:1002A00097200000938000D6130000001300000088
:1002B00083811000930E00006398D1051302120091
:1002C00093022000E31E52FC97210000938181D30A
:1002D0000381010013012000930E2000130E200162
:1002E0006314D103972100009381C1D103810100E0
:1002F0001300000013012000930E2000130E3001A4
:100300006314D101631CC0010F00F00F63000E00E5
:10031000131E1E00136E1E00730000000F00F00F6E
:10032000130E100073000000731000C000000000E6
:1003300000000000000000000000000000000000BD
:0403400000000000B9
:1010000000000000000000000000000000000000E0
:1010100000000000000000000000000000000000D0
:1010200000000000000000000000000000000000C0
:1010300000000000000000000000000000000000B0
:081040000000000000000000A8
:10200000FF00F00F000000000000000000000000D2
:040000058000200057
:00000001FF
